:1000000033C000004EC000004CC000004AC00000D9
:1000100048C0000046C0000044C0000042C00000CC
:1000200040C000003EC000003CC000003AC00000DC
:1000300038C0000036C0000034C0000032C00000EC
:1000400030C000002EC000002CC000002AC00000FC
:1000500028C0000026C0000024C0000022C000000C
:1000600020C000001EC0000011241FBECFEFD4E04E
:10007000DEBFCDBF12E0A0E0B1E0E8E8F2E102C0EF
:1000800005900D92A43BB107D9F713E0A4EBB2E0C1
:1000900001C01D92A03CB107E1F70E949A080C94A0
:1000A0004209AECF0F931F93CF93DF938C01EB01E7
:1000B0008B8181FF1BC082FF0DC02E813F818C810F
:1000C0009D812817390764F4E881F9810193F98348
:1000D000E88306C0E885F985802F0995892B31F4DE
:1000E0008E819F8101969F838E8302C00FEF1FEF49
:1000F000C801DF91CF911F910F910895A0E0B0E06A
:10010000E4E8F0E00C941B09FE01359661917191D1
:100110008091BC039091BD03AF013ED02096E2E0F8
:100120000C9437096091BC037091BD03BBCF0F9352
:100130001F93CF93DF938C01E091BC03F091BD033B
:10014000838181FF21C0C0E0D0E00DC0E091BC03FD
:10015000F091BD0320853185BF01F9010995892BF7
:1001600011F0CFEFDFEFF80181918F01882371F754
:10017000E091BC03F091BD03208531858AE0BF0189
:10018000F9010995892B11F0CFEFDFEFCE01DF9157
:10019000CF911F910F910895ABE0B0E0E2EDF0E058
:1001A0000C940B093C012B015A01FC0117821682A9
:1001B000838181FD03C06FEF7FEFB9C19AE0892E83
:1001C0001E010894211C311CF3012381F20123FD3F
:1001D000859123FF81912F01882309F4A5C18532E0
:1001E00039F423FD859123FF81912F01853221F47C
:1001F00090E0B30157DFE8CF982FFF24EE24992435
:10020000FFE1FF15D0F09B3269F09C3228F4903268
:1002100059F0933291F40EC09D3249F0903369F455
:1002200041E024C052E0F52A84E0F82A28C098E092
:10023000F92A25C0E0E1FE2A22C0F7FC29C0892F57
:1002400080538A3070F4F6FE05C0989C902C1124DF
:10025000980E15C0E89CE02C1124E80EF0E2FF2A6D
:100260000EC09E3229F4F6FC5FC140E4F42A07C0B8
:100270009C3619F450E8F52A02C0983649F4F20188
:1002800023FD959123FF91912F01992309F0B8CF78
:10029000892F8554833018F08052833038F444E03D
:1002A00050E0A40EB51E5FE359830FC0933631F0C2
:1002B000933779F0933509F052C01FC0F501808162
:1002C000898342E050E0A40EB51E610101E010E018
:1002D00011C0F501C080D180F6FC03C06FEF7FEF45
:1002E00002C0692D70E042E050E0A40EB51EC601C8
:1002F0002DD18C015FE7F52213C0F501C080D180BC
:10030000F6FC03C06FEF7FEF02C0692D70E042E0A2
:1003100050E0A40EB51EC6010ED18C0150E8F52A9E
:10032000F3FE06C018C080E290E0B301BBDEEA94A1
:100330008E2D90E008171907B0F30DC0F601F7FCF9
:100340008591F7FE81916F0190E0B301ABDEE11082
:10035000EA94015010400115110581F7E2C094366E
:1003600011F0993661F5F7FE08C0F5012081318161
:100370004281538184E090E00AC0F501808191813F
:100380009C01442737FD4095542F82E090E0A80E51
:10039000B91E9FE6F92257FF09C050954095309548
:1003A00021953F4F4F4F5F4FE0E8FE2ACA01B90148
:1003B000A1012AE030E0D5D0D82ED2183FC0953721
:1003C00029F41F2D1F7E2AE030E01DC01F2D197F4C
:1003D0009F3661F0903720F4983509F0A5C00FC022
:1003E000903739F0983709F09FC004C028E030E01A
:1003F0000AC0106114FD146020E130E004C014FD57
:10040000166020E132E017FF08C0F50160817181BC
:100410008281938144E050E008C0F50180819181A0
:10042000BC0180E090E042E050E0A40EB51EA101C6
:1004300098D0D82ED2188FE7F82EF122F6FE0BC0F6
:100440005EEFF522D91438F4F4FE07C0F2FC05C0C3
:100450008FEEF82202C01D2D01C0192DF4FE0DC033
:10046000FE01ED0DF11D8081803319F499EEF92222
:1004700008C01F5FF2FE05C003C08F2D867809F00B
:100480001F5F0F2DF3FC13C0F0FE0EC01E1510F001
:100490009D2C0AC09D2C9E0C911A1E2D05C080E239
:1004A00090E0B301FFDD1F5F1E15C8F304C01E15E9
:1004B00010F4E11A01C0EE2404FF0EC080E390E0C6
:1004C000B301F0DD02FF1BC001FD03C088E790E02F
:1004D0000EC088E590E00BC0802F867881F001FF88
:1004E00002C08BE201C080E2F7FC8DE290E0B30134
:1004F000D9DD05C080E390E0B301D4DD9A94D9142E
:10050000C8F3DA94F101ED0DF11D808190E0B301A3
:10051000C9DDDD20B1F705C080E290E0B301C2DDA6
:10052000EA94EE20C9F750CEF30166817781CB01C2
:100530002B96E2E18CC6FC010590615070400110E1
:10054000D8F7809590958E0F9F1F0895FC016150FC
:10055000704001900110D8F7809590958E0F9F1FE5
:100560000895FA01AA27283051F1203181F1E89449
:100570006F936E7F6E5F7F4F8F4F9F4FAF4FB1E096
:100580003ED0B4E03CD0670F781F891F9A1FA11D91
:10059000680F791F8A1F911DA11D6A0F711D811D92
:1005A000911DA11D20D009F468943F912AE0269F57
:1005B00011243019305D3193DEF6CF010895462FB6
:1005C0004770405D4193B3E00FD0C9F7F6CF462F97
:1005D0004F70405D4A3318F0495D31FD4052419300
:1005E00002D0A9F7EACFB4E0A695979587957795BD
:1005F0006795BA95C9F700976105710508959B0144
:10060000AC010A2E06945795479537952795BA95CC
:10061000C9F7620F731F841F951FA01D089588E1FD
:100620008093C1008EE08093C20008959B01AC01CD
:1006300060E472E48FE090E0CCD52150304082E05D
:100640008093C0003093C5002093C4000895982F74
:100650008091C00085FFFCCF9093C6000895209143
:10066000C000332727FD30952227330F221F332761
:10067000C9010895CF93DF93EC01F1DF892B19F4C1
:1006800020E030E005C08091C600888321E030E0A2
:10069000C901DF91CF910895289A209A2A9A229A27
:1006A00057985F98299A219A55985D9852985A9828
:1006B0005998519A88EE93E0FC013197F1F7599AD5
:1006C000519A0197F1F75198599A54985C9A429A25
:1006D0003A9A88EE93E028EC30E0F9013197F1F78F
:1006E0000197D9F742983A9A439A3B9A88EE93E059
:1006F00028EC30E0F9013197F1F70197D9F74398E9
:100700003B9A0895E82F2898209A2A98229A2998A7
:10071000219A20E030E060E870E0492F50E0CB0102
:10072000022E02C0959587950A94E2F784239523BB
:10073000892B11F02A9A01C02A98229A89B1299A04
:10074000219A2998219A2F5F3F4F2830310539F798
:100750002A98229A2A98229A2998219A20E030E011
:1007600060E870E04E2F50E0CB01022E02C095955C
:1007700087950A94E2F784239523892B11F02A9A0E
:1007800001C02A98229A89B1299A219A2998219AF6
:100790002F5F3F4F2830310539F72A98229A289A3F
:1007A000209A089581E89AECADDF83E89AECAADFFD
:1007B0008091500290915102A5DF87EF94ECA2DF67
:1007C00080915602909157029DDF80915202909144
:1007D000530298DF81E092E895DF80915402909176
:1007E000550290DF80E598E98DDF81E292E88ADFAB
:1007F00080E197E20197F1F781E892E883DF809149
:1008000050029091510280647DDF81E89AEC7ADF9A
:1008100083E89AEC77DF80E090E074CF0F931F932A
:10082000CF93DF9381E89AEC6DDF83E89AEC6ADF7F
:10083000809150029091510265DF87EF94EC62DF66
:1008400080915602909157025DDF80915202909103
:10085000530258DF81E092E855DF80915402909175
:10086000550250DF80E598E94DDFC0E0D0E000EDB3
:1008700017E081E292E846DFC8010197F1F781E8CD
:1008800092E840DFC8010197F1F72196C431D10504
:1008900081F7DF91CF911F910F9108958F929F92D1
:1008A000AF92BF92CF92DF92EF92FF920F931F937E
:1008B000CF93DF935C01439A3B9AF62E80E886172C
:1008C00010F420E8F22E81E092E81CDF80915002C3
:1008D00090915102806816DF81E292E813DF289838
:1008E000209A2A98229A2998219A20E030E040E81C
:1008F00050E0CA01022E02C0959587950A94E2F74E
:10090000887B11F02A9A01C02A98229A89B1299AE3
:10091000219A2998219A2F5F3F4F2830310549F7B6
:100920002A98229A2A98229A2998219A20E030E03F
:1009300040E850E0CA01022E02C0959587950A94BE
:10094000E2F78A7A11F02A9A01C02A98229A89B18C
:10095000299A219A2998219A2F5F3F4F28303105F3
:1009600049F72A98229AA0E0B0E040E050E0CF2D6D
:10097000D0E021968824992400E810E092E0E92E46
:10098000EF0CCE2CDD2418C14F9B16C1AA2309F011
:1009900086C0B33008F083C0B13031F1B13020F0FF
:1009A000B23009F07AC03EC02A98229A2998219A3A
:1009B00020E030E0C801022E02C0959587950A9488
:1009C000E2F78D729070892B11F02A9A01C02A9853
:1009D000229A89B1299A219A2998219A2F5F3F4F0B
:1009E0002830310539F757C02A98229A2998219A38
:1009F00020E030E0C801022E02C0959587950A9448
:100A0000E2F7847D11F02A9A01C02A98229A89B1CE
:100A1000299A219A2998219A2F5F3F4F2830310532
:100A200049F739C0A4015E25052E0294802D8F70F0
:100A30008527952F9025990F907E8927902D9527B2
:100A4000907F9695052E000C991F569556955695B4
:100A50005F7159275427482F2A98229A2998219A5A
:100A600020E030E0C801022E02C0959587950A94D7
:100A7000E2F78C219D21892B11F02A9A01C02A9836
:100A8000229A89B1299A219A2998219A2F5F3F4F5A
:100A90002830310539F72A98229ABF5F8DC0AF15EB
:100AA00008F03FC0F501EA0FF11D80815827052E9F
:100AB0000294902D9F709527252F2025220F207EB0
:100AC0009227202D2527207F2695052E000C221FFA
:100AD0005695569556955F7152275427492F2A9857
:100AE000229A2998219A20E030E0682F70E0C8010E
:100AF000022E02C0959587950A94E2F786239723E4
:100B0000892B11F02A9A01C02A98229A89B1299A30
:100B1000219A2998219A2F5F3F4F2830310539F7C4
:100B200048C0AF1511F52A98229A2998219A20E0F9
:100B300030E0652F70E0C801022E02C095958795C0
:100B40000A94E2F786239723892B11F02A9A01C091
:100B50002A98229A89B1299A219A2998219A2F5F55
:100B60003F4F2830310539F724C08C179D0719F500
:100B70002A98229A2998219A20E030E0642F70E088
:100B8000C801022E02C0959587950A94E2F7862344
:100B90009723892B11F02A9A01C02A98229A89B1A9
:100BA000299A219A2998219A2F5F3F4F28303105A1
:100BB00039F72A98229AAF5F8A2F90E0C817D90791
:100BC0000CF0E2CE289A209A81E892E89BDD809191
:100BD000500290915102806495DD83E89AEC92DD99
:100BE00043983B9ADF91CF911F910F91FF90EF9027
:100BF000DF90CF90BF90AF909F908F9008951F93FC
:100C0000CF93DF93FC01EB012898209A4F9B75C08E
:100C1000289A209A5D98559A4091B502442381F113
:100C20003091B4022A98229A2998219A20E090E0E3
:100C30002A98229A89B1990F881F8827881F982B94
:100C4000299A219A2998219A2F5F283089F72A9882
:100C5000229AE30FF11D9083132F1F5F1093B402AC
:100C6000141708F445C081E89AEC4CDD5D9A559A5A
:100C700018831092B4021092B50221E030E041C016
:100C80002A98229A2998219A20E090E02A98229A7C
:100C900089B1990F881F8827881F982B299A219A34
:100CA0002998219A2F5F283089F72A98229A1916B5
:100CB0002CF49093B5021092B4021AC05D9A559A22
:100CC00081E092E81FDD81E89AEC1CDD8091500202
:100CD0009091510217DD80915002909151028064F1
:100CE00011DD81E892E80EDD83E89AEC0BDD07C0A8
:100CF0005D9A559A2FEF3FEF04C0289A209A20E082
:100D000030E0C901DF91CF911F9108951F93182FF3
:100D10008A3011F48DE0FADF812F99DC80E090E0D9
:100D20001F9108951F93182F8A3011F48DE0FADF78
:100D30002A98229A2998219A20E030E060E870E011
:100D4000412F50E0CB01022E02C0959587950A9461
:100D5000E2F784239523892B11F02A9A01C02A985F
:100D6000229A89B1299A219A2998219A2F5F3F4F77
:100D70002830310539F72A98229A80E090E01F91B7
:100D800008950F931F93DF93CF930F92CDB7DEB7E4
:100D900008EC10E00BC080E091E06DE07FDD88EEB4
:100DA00093E0F8013197F1F70197D9F758DC892BD7
:100DB00091F3CE0101965EDC0F90CF91DF911F91F0
:100DC0000F9108958F929F92AF92BF92CF92DF9230
:100DD000EF92FF920F931F93DF93CF9300D0CDB785
:100DE000DEB700E010E0EE245AE0F52E42E0842E5B
:100DF000912C8C0E9D1EAA24BB246E010894C11C4C
:100E0000D11C03C000E0EE24E394112381F44C993B
:100E100007C08EE091E066E041DD3AE0F32E07C0C6
:100E2000FF2029F0FA9485E191E066E037DD8AE35E
:100E300093E0B401E4DE2FEF8F3F920721F001979A
:100E400009F05EC004C0429A3A9A11E059C0429833
:100E50003A9A8A81482F50E04250504090E01EC09C
:100E6000E65CFC4F808195013827032E0294802D8B
:100E70008F708327632F6025660F607E8627602D25
:100E80006327607F6695032E000C661F36953695A6
:100E900036953F7136273227282F9F5FE92FF0E0E4
:100EA000E417F507ECF26091BC037091BD038BE78A
:100EB00090E0F8D810E00AC0E65CFC4F6091BC03FB
:100EC0007091BD03808190E0EDD81F5FE12FF0E0CD
:100ED0008A8190E00297E817F90774F36091BC03E8
:100EE0007091BD038DE790E0DDD883E89AEC0ADCD1
:100EF0006091BC037091BD038AE090E0D3D810E00C
:100F0000AEDB892B09F481CFC601B4DB8981883738
:100F100089F0893728F48B3169F0813769F40AC088
:100F20008B3709F46FCF8D3739F48AEB92E0602F5D
:100F3000B5DC6BCFEE2049F007FD67CFE02FF0E086
:100F4000E654FD4F80830F5F60CF0F900F90CF91DD
:100F5000DF911F910F91FF90EF90DF90CF90BF90A6
:100F6000AF909F908F900895AF92BF92CF92DF92F3
:100F7000EF92FF921F93DF93CF9300D0CDB7DEB7F0
:100F8000E2E0AE2EB12CAC0EBD1E7CE1C72E71E0AE
:100F9000D72E6AE3E62E61E0F62E46C08AE393E0A0
:100FA000B5012DDE2FEF8F3F920721F0019709F059
:100FB0003BC008C06091BC037091BD038EE290E01D
:100FC00071D832C000D000D0EDB7FEB73196ADB7C2
:100FD000BEB71296DC92CE9211978A8182831382D9
:100FE0008DD810E014C000D000D0EDB7FEB7319618
:100FF000ADB7BEB71296FC92EE921197A12FB0E05A
:10100000A65CBC4F8C918283138278D81F5F0F90AF
:101010000F900F900F908A81181728F38AE090E0C4
:1010200081D883E89AEC6EDB1ADB892B09F4B6CF02
:10103000CE0101961FDB0F900F90CF91DF911F9192
:10104000FF90EF90DF90CF90BF90AF900895CF9238
:10105000DF92EF92FF920F931F93DF93CF930F9244
:10106000CDB7DEB7F0E4CF2EF1E0DF2E7E0108949D
:10107000E11CF11C03E411E04EC000D0ADB7BEB7D7
:101080001296DC92CE92119739D80F900F90E7DA32
:10109000892BE9F3C701EEDA892B09F43CC000D0B3
:1010A00000D0EDB7FEB73196ADB7BEB712961C9320
:1010B0000E93119789818283138220D80F900F900D
:1010C0000F900F9089818B3609F18C3628F48F337D
:1010D00041F08236E9F418C08237A1F08437C1F4B8
:1010E0000FC087E491E023D881E691E020D888E81A
:1010F00091E01DD883EB91E01AD885ED91E00AC00C
:1011000040DE09C031DF07C089DB05C05BDE03C0FC
:101110008EEF91E00CD880917402882309F0ADCF56
:101120000F90CF91DF911F910F91FF90EF90DF9083
:10113000CF9008950F931F93DF93CF930F92CDB766
:10114000DEB7F89454985C9A439A3B9A43983B9A3A
:1011500066DA60E875E280E090E068DA88E592E0BF
:101160009093BD038093BC0300D000D08EE092E04A
:10117000EDB7FEB79283818385E792E09483838302
:101180000E947E00299A219A2A9A229A289A209AC5
:1011900057985F980F900F900F900F907DDA02DBB9
:1011A0008E010F5F1F4FC80165DA892BE1F78BE1D4
:1011B00092E060E073DB06DE8CE192E00E94970033
:1011C00046DF80E090E00F90CF91DF911F910F916B
:1011D0000895A1E21A2EAA1BBB1BFD010DC0AA1F78
:1011E000BB1FEE1FFF1FA217B307E407F50720F090
:1011F000A21BB30BE40BF50B661F771F881F991F0B
:101200001A9469F760957095809590959B01AC0153
:10121000BD01CF0108952F923F924F925F926F923E
:101220007F928F929F92AF92BF92CF92DF92EF9276
:10123000FF920F931F93CF93DF93CDB7DEB7CA1BF7
:10124000DB0B0FB6F894DEBF0FBECDBF09942A8822
:10125000398848885F846E847D848C849B84AA84CA
:10126000B984C884DF80EE80FD800C811B81AA8157
:10127000B981CE0FD11D0FB6F894DEBF0FBECDBF22
:08128000ED010895F894FFCF81
:1012880048656C6C6F2C20726164696F2100525E36
:101298002A7C423100525E2A7C42300052656365E6
:1012A80069766564207061636B6574206F66206C75
:1012B800656E6774682025640A002530327820003E
:1012C8003E200025630A003F097072696E7420741D
:1012D8006869732068656C70206D657373616765F4
:1012E80000620962757A7A206F6E2052462028358E
:1012F800303020487A204F4F4B20666F72203230B2
:10130800206379636C657300720972656365697639
:101318006520616E64207072696E74207061636B01
:1013280065747320756E74696C206B65797072656D
:1013380073730074097472616E736D6974207061DF
:10134800636B65747320756E74696C206B65797056
:1013580072657373006B0972656D6F7465206B65D8
:1013680079666F622064656D6F206C6F6F70207591
:101378006E74696C206B6579707265737300756E35
:101388006B6E6F776E20636F6D6D616E64000A2AF5
:101398002A2A202573202A2A2A0A00002A2A2A20F3
:1013A800656E746572696E6720636F6D6D616E64DA
:1013B80020696E7465727072657465723B20747909
:1013C800706520273F2720666F722068656C700063
:1013D800138023C6819440A600000002000000008C
:1013E80086060000000000000002000000009206CF
:1013F800000000000168722E63202D2048656C6C87
:101408006F20526164696F2076302E32204D6179E9
:1014180020203220323031312031373A35343A34D5
:101428003400303132333435363738394142434469
:041438004546000025
:00000001FF
